:1000000000308A007B280000FF00030E8301A1005E
:100010007F08A0000A08A8008A01A00E0408A20018
:100020007708A3007808A4007908A5007A08A6003C
:100030007B08A700831383128C308400801D222844
:100040008C193528220884002308F7002408F800BA
:100050002508F9002608FA002708FB0028088A006E
:10006000210E8300FF0E7F0E09008A114528130818
:100070003008930014168C118316141C4128831227
:100080003C28F80183128A1168288316850183129F
:1000900085018316941A51288312AA011318AA17EE
:1000A000831683122A08AA0AAF002F087F3C031C7C
:1000B0006128831614185E288312592883121308A6
:1000C000A9002F08803C031D68282908B0003728A4
:1000D0008C118A1122280830AD02031C7A282D3099
:1000E00084000310800C000803197A287828000087
:1000F000800B7728003484011F308305703083160D
:100100008F0006168614A2309300363083129400B6
:1001100083161F129F121B0880399B0007309C001A
:1001200003308312AA0083161F129F121B08803906
:100130009B0083121F1083160108C03981000B3009
:10014000F700073083128101813084000008F03904
:100150000738800064000008F739F719F039770490
:10016000800090010030F800920000308316920069
:1001700007309C0005080630F700F70BBD2800008B
:100180001C0883120D1383169D0172308F00C0303E
:1001900083128B0483168C1580308312A9002908E2
:1001A000803C031DD8288316850183128501CF2842
:1001B0007F302907AB00831685011230831285003A
:1001C0002B08AD006B20831685018312850100008A
:1001D00000006400831685010C30831285002B0813
:1001E000FE3CAC00AD006B208316850183128501B7
:0801F00000000000CF286300AD
:04400E00343FFC3F00
:00000001FF
